:020000001828BE
:080008009000900E030E910020
:10001000040E92000A0E93000B1D10280B112E21C6
:10002000130E8A00120E8400110E8300100E0900B8
:100030008316C030810083120B08DF398B00A301C7
:10004000A4010030A9002308AA000030AB00C8209A
:100050000130A9002408AA000030AB00C820A70185
:10006000A20183160108F8390438810083120B08B5
:10007000DF39A0388B006430220203188C2800304E
:10008000A9002308AA000030AB00C8200130A90055
:100090002408AA000030AB00C820831605081038D9
:1000A0008500831205081039A8000F30280201309E
:1000B00003180301FF390130031D0030003C031D0C
:1000C00062283F280030A9002308AA000030AB00B6
:1000D000C8200130A9002408AA000030AB00C820C5
:1000E0008316050810388500831205081039A8000A
:1000F00028080F3C013003180301FF390130031DAC
:100100000030003C031D852862288D012708013E30
:1001100003188D0AA7003B280B08DF398B00083035
:100120008D008E0127088F0003108F1B03148E0D86
:100130000A308E0203189E288E0703108F0D8D0B38
:1001400094280F08A40008308D008E0127088F0026
:1001500003108F1B03148E0D0A308E020318B22871
:100160008E0703108F0D8D0BA8280F082702A30000
:100170000030A9002308AA000030AB00C8200130DD
:10018000A9002408AA000030AB00C8202F28C728E7
:10019000083094000430950002309600013097003A
:1001A000C0309800F9309900A4309A00B0309B001C
:1001B00099309C0092309D0082309E00F8309F0064
:1001C0008030A0009830A10008308D008E012A08F0
:1001D0008F0003108F1B03148E0D0A308E0203183C
:1001E000F3288E0703108F0D8D0BE9280E08183E9B
:1001F00084000008AC00003029020130031C030118
:10020000FF3903190C292908033C0130031C0301A1
:10021000FF3903190C290130003C03192D298316DD
:100220000508F039850006080039860083120508A4
:10023000F03985002B08003C031920297F30AC05DC
:10024000060800392C0486000508F0398D002908BD
:10025000143E840000080D04850008008C0122086B
:0A026000013E03188C0AA2000800FA
:00000001FF
